:0600000075817F0200265D
:100023000201E87545007547017544007543007585
:1000330090FF1201D5753400753500752E00752FAC
:1000430000753000753100753200753300D2B2C2CD
:1000530004D208D207D205D209C20DD2127400907D
:100063000010F0900011F0900012F0900013F09047
:100073000014F01211FE1212331202C81202C82029
:10008300B2FD12011B1202DCE53FB400061200A50B
:10009300020088B401061200D40200881200E802AC
:1000A300008830071420B2FD7452120202745812F1
:1000B300020212011BC207D20520920C1201083062
:1000C30005051201A5C20522200505120190D205DE
:1000D30022300805120A9DC208209206120A76C22F
:1000E3000522D20522300908120A9D754600C2096D
:1000F300120A64300C0C120B53120B8DC205121230
:100103003322D20522120E98120990120FDF121118
:100113000D120CB3120E6A22745C120202743012B6
:1001230002021201907438120202744A120202741B
:1001330030120202744E120202120FFD74311202C7
:10014300027434120202744A12020274311202025D
:100153007435120202744E120202743112020274D6
:1001630035120202744A1202027431120202743509
:10017300120202744E1202027436120202744A12FE
:1001830002027430120202744E12020222743712F7
:100193000202744A1202027430120202744E1202F4
:1001A30002227437120202744A120202747F12018D
:1001B300BD12024A744E12020222F52E752F0075EB
:1001C3003201753300782E7932120844868208860C
:1001D3008322C2AF438780759B1F759AD975985048
:1001E300D2ACD2AF22C0D0C0E020980A30990BC263
:1001F30099C2000201FDC298E599D0E0D0D0322027
:1002030093FDF599D2002000FD2275F00A84AFF02A
:1002130075F00A842430120202E5F024301202023F
:10022300EF24301202022275F00A84AFF0EF24307B
:10023300F62275F00A84AFF075F00A84E5F02430F5
:10024300F6EF243008F622C0E0E8C0E0C2D5AA8267
:10025300AB837C107D271202A860042430D2D57CA6
:10026300E87D031202A8700330D50724301202027E
:10027300D2D57C647D001202A8700330D5072430E8
:10028300120202D2D5EAABF075F00A84700330D5BE
:10029300052430120202E5F08BF02430120202D062
:1002A300E0F8D0E022780008C3EA9CFAEB9DFB500B
:1002B300F618EA2CFAEB3DFBE822783279FF0000CE
:1002C300D9FCD8F822784B79FF0000D9FCD8F82262
:1002D300780A7996D9FED8FA22209108753F00D280
:1002E30009D20822309008753F01D209D20722753E
:1002F3003F02D207D20822FD90190693FFA3ED9384
:10030300FE22FD9018D693FFA3ED93FE22B5400382
:10031300020319754600F540B43B0302032640FB74
:1003230002041E75F004A490032E7390127A229097
:1003330012B0229012E9229012FB229012FF229017
:100343001303229013072290130B22901310229071
:1003530013152290131B2290131E22901323229015
:1003630013282290132F22901332229013382290B5
:10037300133A2290133F2290134322901346229064
:10038300134A2290134F2290135322901355229015
:0E039300135D229013672290136C2290137159
:1003A100229013772290137D229013882290138E2E
:1003B100229013962290139F229013A5229013ACA2
:1003C100229013B2229013B9229013BF229013C826
:1003D100229013CE229013D2229013D7229013DCB5
:1003E100229013E3229013EB229013F72290140032
:1003F1002290140522901412229014182290141E97
:1004010022901422229014292290142D2290143229
:1004110022901438229014452290145122C3943C06
:1004210075F004A490042973901457229014632248
:1004310090146A22901470229014752290147822DC
:1004410090147E229014882290148E22901493226C
:1004510090149A2290149E229014A2229014A72202
:100461009014B2229014B7229014BC229014C1228D
:100471009014C8229014CD229014D2229014D72225
:100481009014E1229014E5229014EB229014F022B2
:100491009014F3229014F92290150222901508224B
:1004A10090150E22901513229015182290151D22D9
:1004B10090152122901524229015292290152E2283
:1004C10090153122901534229015382290153B2237
:1004D100901540229015452290154A2290154D22E3
:1004E10090155022901555229015582290155B2297
:1004F100901560229015652290156A229015702240
:1005010090157422901578229015822290158722D9
:1005110090159322300E0785418285428322121164
:10052100FE12126A12059975F006A49005307390B7
:10053100159B02059090159E0205909015A002054D
:10054100909015A80205909015AF0205909015B6F0
:100551000205909015BD0205909015C2020590907C
:1005610015C90205909015D20205909015D6020585
:10057100909015DD0205909015E30205909015ED20
:100581000205909015FA02059090160D02059085CE
:100591008241858342D20E22B40503C2112240FB5F
:1005A100D21122300E07854182854283221211FE2B
:1005B10012126A75F006A49005BC7390161C02060F
:1005C1001C90162602061C90162A02061C90163450
:1005D10002061C90163902061C90163E02061C905B
:1005E100164A02061C90165402061C901658020662
:1005F1001C90166102061C90166502061C90166F6F
:1006010002061C90167602061C90168002061C90AB
:10061100168A02061C90169202061C858241858369
:1006210042D20E22300E0785418285428322121169
:10063100FE12126A75F006A490063D73901696029A
:10064100069D9016A102069D9016A602069D901683
:10065100B102069D9016B702069D9016BD02069D39
:100661009016CA02069D9016D502069D9016DB02D1
:10067100069D9016E502069D9016EA02069D9016CB
:10068100F502069D9016FD02069D90170802069D33
:1006910090171402069D90171D02069D85824185C3
:1006A1008342D20E22300E07854182854283221277
:1006B10011FE12126A75F006A49006BE73901722FD
:1006C10002071E90172D02071E90173202071E9077
:1006D100173702071E90173B02071E9017420207A9
:1006E1001E90174C02071E90175202071E901756B4
:1006F10002071E90175C02071E90176202071E90E8
:10070100176802071E90176E02071E9017760207E0
:0E0711001E90177E02071E90178502071E8598
:10071F008241858342D20E22300E07854182854267
:10072F0083221211FE12126A75F006A490073F730E
:10073F0090178C02079F90179202079F90179C02A9
:10074F00079F9017A802079F9017B302079F901754
:10075F00BB02079F9017C102079F9017C702079F01
:10076F009017D302079F9017DE02079F9017EB0297
:10077F00079F9017F102079F9017F902079F901795
:10078F00FF02079F90180402079F90181002079FFF
:10079F00858241858342D20E22300E0785418285A4
:1007AF004283221211FE12126A75F006A49007C03E
:1007BF007390181702082090181F02082090182312
:1007CF000208209018260208209018320208209064
:1007DF00183E02082090184902082090185102086C
:1007EF002090185B02082090185F02082090186470
:1007FF0002082090186A02082090186F02082090B3
:10080F00187702082090187C02082090188A020896
:10081F0020858241858342D20E22E627F5230809DF
:10082F00E637F524782322C3E697F5230809E697E0
:10083F00F524782322862387250809862487261204
:10084F0008C9782822862808862908862A08862B30
:10085F00872509872612086C7823792A22752C00A0
:10086F00752D101208AE12087F1208A2D52DF42292
:10087F00C3E52A9525E52B9526E52C9400500122FA
:10088F00E52A9525F52AE52B9526F52BE52C9400E1
:10089F00F52C22B3E52333F523E52433F52422C3C6
:1008AF00E52833F528E52933F529E52A33F52AE537
:1008BF002B33F52BE52C33F52C22E5238525F0A4DE
:1008CF00F52885F029E5248526F0A4F52A85F02B57
:1008DF00E5248525F0A42529F529E52A35F0F52A03
:1008EF00E52B3400F52BE5238526F0A42529F529E2
:1008FF00E52A35F0F52AE52B3400F52B227A0FC2C5
:10090F0095D294A29633C933C9C294DAF2F8D2952C
:10091F0022D2957A0574E0C294C295339297D294FD
:10092F00DAF512090C8836893753370F22D2957AA8
:10093F000574E8C294C295339297D294DAF51209EE
:10094F000C8838893953390F22D2957A0574F0C241
:10095F0094C295339297D294DAF512090C883A899A
:10096F003B533B0F22D2957A0574F8C294C295334C
:10097F009297D294DAF512090C883C893D533D0FBA
:10098F002212092085362E85372F753000753100DC
:10099F00782E75320A7533007932120829862E089F
:1009AF00862F753000753100782E75320A75330039
:1009BF007932120844753255753301793212085461
:1009CF00E675F002A4F5492212092085362E8537E7
:0909DF002F753000753100782EEF
:1009E80075320A7533007932120829862E08862F47
:1009F800753000753100782E75320A7533007932FA
:100A08001208447532557533017932120854E612CA
:100A180011DF75F002A4120305EE22120974853C59
:100A28002E853D2F753000753100782E753214757E
:100A380033007932120829862E08862F7530007502
:100A48003100782E75320A753300793212084475F0
:100A580032557533017932120854E62220920C205F
:100A68000D08D20CD20DD20AD20B22C20D2220B20E
:100A7800FD7415120202120AFE7417120202120BFA
:100A8800317416120202120B4C7407120202120A77
:100A9800E61202BD22745212020274581202027443
:100AA8001412020274001202027415120202747FF8
:100AB8001202027417120202120B31741612020289
:100AC800120B4C740712020274AD1202021202BD1C
:100AD80020B2FD7414120202747F12020222120A5A
:100AE800232480120AF51211B012020222B4F6036E
:100AF80024062250FB22120958853A82853B83E559
:100B080082C4540FF9E583C46975F00284120202A5
:100B180022120958853A82853B83E582C4540FF92D
:100B2800E583C46975F002842212093C8538828500
:100B38003983E582C4540FF9E583C46975F01184DB
:100B4800120202221209D71202022274151202029C
:100B5800120AFE7417120202120B317416120202E4
:100B6800120B4C740712020222120974853C82850A
:100B78003D83E582C4540FF9E583C46975F00284A6
:100B880022120A2322300C08209205120B89F548FC
:100B9800E548B47711300B08754600754701C20B5C
:100BA800120BD7D20A2250ED300A05754600C20A48
:100BB800120BBED20B22120310E54693700B75463A
:100BC80000C20CC20D20B2FD22054612020222E527
:100BD80047B40104120BF922B40204120C1822B40F
:100BE8000304120C4022B40404120C5F22120C8875
:100BF80022120515E5469370117546007404120219
:100C080002754702C20E20B2FD22054612020222D8
:100C18002011061205A4020C24120625E54693703D
:100C2800117546007404120202754703C20E20B201
:100C3800FD220546120202221206A6E5469370110D
:100C48007546007404120202754704C20E20B2FDF4
:100C580022054612020222120727E54693701B75E9
:100C68004600740612020274061202027406120288
:100C780002754705C20E20B2FD2205461202022265
:100C88002092151207A8E54693701A754600740657
:100C98001202027406120202754701C20CC20DC28A
:100CA8000E20B2FD2205461202022212093C8538A6
:100CB80082853983120D95F5387431120202743425
:100CC800120202744A120202E53875F00884121101
:100CD80062120D4D12024A744E120202743112024F
:100CE800027435120202744A120202E53875F008DD
:100CF80084121162120D4D12024A744E12020274CD
:100D080034120202744A120202E538120D6B120202
:100D18004A744E1202027435120202744A12020216
:100D2800E538120D5312024A744E1202027436123A
:100D38000202744A120202E538120D4D12024A7478
:100D48004E12020222F58275830022F52E752F00BD
:0E0D5800753207753300782E79321208448602
:100D66008208868322F52E752F00753207753300AB
:100D7600782E7932120844752E9F752F0F86320809
:100D86008633782E7932120836868208868322E5E3
:100D960082C4540FF9E583C46922743812020274BE
:100DA6004A1202027440120D4D12024A744E120289
:100DB600027430120202744A120202E53A120D4D12
:100DC60012024A744E120202227438120202744A45
:100DD60012020274C1120D4D12024A744E12020220
:100DE6007430120202744A120202E53A75F002A445
:100DF600120D4D12024A744E120202227438120269
:100E060002744A12020274C0120D4D12024A744E46
:100E16001202027430120202744A120202E53A7594
:100E2600F0FFC5F0C395F075F002A4120D4D120245
:100E36004A744E120202227438120202744A1202D4
:100E4600027403120D4D12024A744E1202022274EB
:100E560030120202744A1202027430120202744EF6
:100E660012020222120958853A82853B83120D9599
:100E7600F53A7007120E3D1201A52279FFC9C399F2
:100E8600F53AB48003020E945004120DCF22120ECE
:100E96000222120974853C82853D83120D95F53C2C
:100EA60075F00284120EAE22B4020FD20F754E01F7
:100EB600754B00754C00754D002240EFC20FB4080B
:100EC6000D754E02754B0E754C08754D002240F19E
:100ED600B4100D754E03754B18754C0E754D0822E2
:100EE60040F1B4180D754E04754B20754C18754DB0
:100EF6000E2240F1B41E0D754E05754B12754C0849
:100F0600754D002240F1B4250D754E06754B1675CC
:100F16004C08754D002240F1B42B0D754E07754BEC
:100F26000E754C06754D002240F1B4310D754E0814
:100F3600754B18754C0E754D062240F1B4370D757C
:100F46004E09754B12754C06754D002240F1B441A1
:100F56000D754E0A754B16754C06754D002240F1FF
:100F6600B44B0D754E0B754B14754C0A754D00221E
:100F760040F1B4540D754E0C754B10754C08754DFB
:100F8600002240F1B45D0D754E0D754B0C754C0687
:100F9600754D002240F1B4670D754E0E754B0E75FA
:100FA6004C0A754D002240F1B4700D754E0F754B0D
:100FB6000E754C04754D002240F1B47D0D754E1032
:100FC600754B14754C0E754D002240F1754E11751A
:100FD6004B30754C18754D0022E549600C301205F2
:100FE600120FFDC212120FF5221210C1D21222E503
:100FF6004EB54F0122F54F300F0712108E12101208
:101006002212103112105012106F22227431120265
:10101600027431120202744A12020274331202027C
:101026007430120202744E1202022274311202024B
:101036007431120202744A120202743112020274EC
:1010460030120202744E120202227431120202742B
:1010560032120202744A120202743112020274300F
:10106600120202744E120202227431120202743308
:10107600120202744A12020274311202027430120F
:101086000202744E120202227431120202743212E9
:101096000202744A1202027430120202744E1202E2
:1010A6000274311202027433120202744A120202EC
:1010B6007430120202744E120202227431120202BB
:1010C6007431120202744A1202027430120202745D
:0E10D6004E1202027431120202743212020231
:1010E400744A1202027430120202744E1202027422
:1010F400311202027433120202744A120202743070
:10110400120202744E120202221211741202FA74B2
:1011140031120202744A1202028E828F8312024A30
:10112400744E1202021211941202FA743212020262
:10113400744A1202028E828F8312024A744E120281
:10114400021211A21202FA7433120202744A120237
:10115400028E828F8312024A744E12020222B40F4C
:1011640001224002740F22B4C00122400274C02242
:10117400C374C0954BF53EE54912116BB53E0302AD
:1011840011884007E53E254BD21022254BC2102280
:10119400201005E549254C22C3E53E254C222010AC
:1011A40005E549254D22C3E53E254D22C3B4FD0185
:1011B40022400374FD22C3B48001225002748022B1
:1011C400B4F00122400274F022B478012240027487
:1011D4007822B43001224002743022C3B447012281
:1011E4004002744722900010E004B410027400F02E
:1011F400900000A98229F582E022900014E0FA9080
:101204000011E004B40F0274FFF0901891932A9037
:101214000014F0900013E004B410027400F0F9908C
:101224000014E0FA900000E58229F582EAF02290A9
:101234000014E0FA900012E004B4110274FFF0907C
:1012440018A0932A900014F0121217221211E954D4
:101254000160081211E9541F246022747F221211C4
:10126400E975F02084221211E975F010842212111C
:10127400E975F01F84228B878D0606BF8B8B0606CB
:10128400BE94800606BA899906BA8780BA06BB81DD
:10129400C4BB06BB83A6818D069ABF06068D8780D4
:1012A4008D06BF838D8D060606060600BF838D8DD1
:1012B400068D87808D069ABF0606BB83A6818D06A0
:1012C400BB81C4BB06BA8780BA06BA899906BE94A4
:1012D400800606BF8B8B06068B878D0606A795A412
:1012E400060606060081B606AA818D069B8D05AA10
:1012F4009691808D9606008B878D00BF8B8B00BEE8
:10130400948000BA899900BA8780BA00BB81C4BBB3
:1013140000BB83A6818D009ABF008D87808D00BF9E
:10132400838D8D00809183A6818D008780008780C6
:1013340006848C00A000A00698060081BFBB008E26
:10134400A3008E89BF00AFA48EBF00838EBF009917
:1013540000C69183BDBE81C2009F82C4BE94898EA3
:1013640081C200919AA79600A6848096008CC6A09C
:10137400BF9600949AB080A400C094838DBB8C81E6
:10138400BD818D009489AD89BF00B283A789918006
:101394008D0083088D07960FA580008C83B6808D01
:1013A40000A781BBBF818C0083BF818CBB00A0BF21
:1013B40094898DBB009906AA81BF00BB83BF81922B
:1013C4008480BF009489C581BF00AA808C00BA9133
:1013D4008480008CA28D8D00A08D80A696BC00B266
:1013E400839183C4BB8000AA9184C21E0FB8A491C8
:1013F4001E0F009181BABF0689BA0600B280BF9859
:1014040000A7818DBF8106BB8780A7960600AE9496
:10141400878CBB00BBBF81C4BB00AA9ABB00BBBF07
:1014240094818FBB00AB919A00BBBF89C7008CA08D
:10143400A781C200948706C3068D8D069489910600
:1014440000C78790C5068CA0A781C20600BF83C5CC
:0E1454008DA400AF828DBB068CA0A781C206BE
:1014620000C3898DA897BF00BF80BD97BF00BA8314
:101472008DC100B6A400C3888C81C200BFBB81B4F9
:10148200829482BFBB00AF9487C5BB00BB83C4BB41
:10149200008C81BBBF968000C7A3960083949900FD
:1014A200AE94808C00BB848E8EBDB687808D8D00FD
:1014B200BA91A39600A689BF9400949A8D8D00A438
:1014C200BCBC818D8D00C392A3C100BBC3878000C9
:1014D200A69791B000A6888EAE96BA8A8A9200B27A
:1014E200969100A68B8C818D00919AAE8000AB9C68
:1014F200008C83838D8D009484BBBF848C878D0088
:10150200BB81BBBF9600AA9487A796008C87A7963B
:1015120000BA87A796009281C6BC008780BB00B73D
:101522009600AB87AE8000A406C29A009EBB008ED6
:10153200A400AEA38E0084B5009183BABF00948745
:1015420080BF00BF86948D00888E0088BA00878D88
:10155200AE9600818E00B89500A6948890008D8783
:1015620080BB00C38B8B9100BBBF998C8000BA9467
:101572008000A492BF00BF89C50681ABA3BF06004D
:10158200C69180A70084809104AA8004AA82C4051F
:1015920000BE838FC506A00600878000A000BF9909
:1015A2008D9AAFA4BB008CC6A0BF96BB008C848F63
:1015B200C280BB009489AD89BFBB009FA681BB00DE
:1015C2008EA4AB85AE8000BBC38780A699C296006D
:1015D200B387BF00918ABB81BA96008C8484848CC5
:1015E20000BBAC8480AE968C838D00A78106BF972A
:1015F2008C818D9ABF940500A781068C98BBBF96FB
:1016020088BAA08D8106A696A706008C81BBBF96DC
:10161200C69483A780AE828EBF00BF89C50581AB09
:10162200A3BF0500AB919A00B3A405BF8B05BE8191
:101632000500BBBF89C7009187BABA00BA8480BFD0
:1016420081B29A8DBBBF0500BB8C9F06918480C47A
:101652000600BB97B600AE94808C0688BA0600B727
:101662009ABF00AA819180BA06818E0600AE83BB22
:10167200BF949C00A6948480AE0588BA0500AA9403
:101682009AC405BE948B0500918AC40583BF0500E8
:10169200C2819200BF89C5BB0581ABA3BF0500AB68
:1016A200919ABB00B3A4BB05BF8B05BE810500BBED
:1016B200BF89C7BB009187BABABB00BA8480BFBBDF
:1016C20081B29A8DBBBF0500BB8C9FBB0691848003
:1016D200C40600BB97B680BB00AE94808CBB068864
:1016E200BA0600B79ABFBB00AA819180BABB068135
:1016F2008E0600AE83BBBF949CBB00A6948480AED2
:10170200BB0588BA0500AA949AC4BB05BE948BBBDC
:101712000500918AC4BB0583BF0500C28192BB004C
:10172200818DC29482AF81AA8191008D8780BB0096
:10173200C38B8B9100BA948000BA9AAA9F81BB0096
:10174200A6888EAE96BA8A8A9200BBBF998C800018
:10175200AF98C500BA848FC280008C81BBBF800065
:10176200AE838C8DBF008C8480AE8000AE828C8173
:10177200BFB6C200AE9A8DA89586BB00C087C5A72A
:1017820081C4008C99AE9686BB00AF9487C5BB001E
:10179200BFBB81B4829482BFBB00BC81BF80059174
:1017A2008780BF800500C2949AA780B899BB81BB8D
:1017B20000B2839183C4BB8000B280BF98BB00BAE1
:1017C20091A396BB00C78790C5058CA0A781C205CF
:0E17D20000AA9183C506AF89C506BB00A7819A
:1017E0008DBF8106BB8780A796BB00AA949A8DBB4C
:1017F00000AA818E828E84BB00BA9ABB81BB00C3D3
:1018000092A3C100AF828DBB068CA0A781C2060047
:10181000BF80BD97BFBB00AA8006C299A706008300
:101820008EBF00990600878005AFA48EBF058EA4E9
:101830000500060606838D80939A060606000606B6
:101840008480048C808E06060006A406C29A0606D2
:1018500000AA80BB8480B1BB060600BBA40600A61C
:101860009F060600918480C40600AB86BF060082F6
:10187000C4BFB69F800600A684809F00A689BF04CF
:1018800082A696048C838D0606008E9A8C91800623
:101890000003002C0C01057E2133E6FF0B4D68147C
:1018A0006405140D004B1A26351E1A96114042C8C5
:1018B000C921232527292C2E3134373A3E41454969
:1018C0004E52575D62686E757B838B939CA5AFB952
:1018D000C4D0DCE9F7F700000000000000010002BE
:1018E00000030004000500060006000700070008CA
:1018F000000800090009000A000A000B000C000C97
:10190000000D000E000F0010001100120013001453
:10191000001600170018001A001C001D001F0021EF
:101920000023002500270029002C002E0031003460
:101930000037003A003E004100450049004E005289
:101940000057005C00630068006E0075007C008337
:10195000008B0093009C00A500AF00B900C400D02C
:1019600000DC00E900F70106011501260137014AF4
:10197000015D01720188019F01B801D201EE020BE5
:10198000022A024B026E029302BA02E40310033FE2
:10199000037003A403DC04170455049704DD052732
:1019A000057505C80620067D06E0074907B8082D1D
:1019B00008A9092D09B90A4D0AB00B900C400CFA80
:1019C0000DC00E910F6F0F6F464C414D4520544195
:1019D0004C4B494E472D53594E54482D4D4F44556D
:1019E0004C45204555524F205241434B20564552BD
:1019F00053494F4E202D203230313120564552531D
:101A0000494F4E20312E30302028632962792061E1
:051A10006D70657265B8
:00000001FF
